:030000000205599D
:0C055900787FE4F6D8FD75815C0205A0F7
:1008810002440000024600000C4800000000000085
:100891000000000000000A3A303132333435363777
:0E08A1003839015C000154090155090156095E
:10084B001208B012096E7F801209307F4E1209B761
:10085B007F811209307F551209B77F821209307FD1
:10086B004D1209B77F831209307F3A1209B7120074
:06087B000312045380F893
:1008D300D3EF9400EE940040137D017C8E7B02DB0A
:0C08E300FEDCFADDF6EF1F70E71E80E47B
:0108EF0022E6
:10000300E4F508F509F50AF50B30B4030201607F46
:1000130064FE1208D330B4030201607F0112093079
:100023007B007A0079367F521206E0EF600302010B
:1000330060FB7A007957120665EF60030201607F67
:10004300C01209307F571209B77FC11209307F49A7
:100053001209B77FC21209307F541209B7E4F508B9
:10006300F509E50925E0FEE42400FFEE3420FE1245
:1000730008F0EFF4600302014AE50925E0FEE424F9
:1000830001FFEE3420FE1208F0EFF4600302014A90
:10009300E50925E0FEE42402FFEE3420FE1208F019
:1000A300EFF4600302014AE50925E0FEE42403FFBF
:1000B300EE3420FE1208F0EFF4600302014AE50972
:1000C30025E0FEE42400FFEE3420FEAD5712094084
:1000D300E50925E0FEE42401FFEE3420FEAD5812CD
:1000E3000940E50925E0FEE42402FFEE3420FEADDD
:1000F30059120940E50925E0FEE42403FFEE34200C
:10010300FEAD5A1209407FC01209307F571209B75A
:100113007FC11209307F491209B77FC21209307FAC
:10012300541209B77FC31209307F4F1209B77FC436
:100133001209307F201209B77FC51209307F4B1295
:1001430009B712092780160509E50970020508C3D6
:100153009408E50864809480500302006530B50379
:100163000202787F647E001208D330B5030202785E
:100173007F011209307B007A0079367F521206E044
:10018300EF6003020278FB7A007957120665EF608D
:10019300030202787FC01209307F431209B77FC17F
:1001A3001209307F4C1209B77FC21209307F451202
:1001B30009B7E4F50AF50BE50B25E0FEE42400FF9F
:1001C300EE3420FE1208F0EF65576003020262E589
:1001D3000B25E0FEE42401FFEE3420FE1208F0EFCD
:1001E3006558707BE50B25E0FEE42402FFEE342026
:1001F300FE1208F0EF65597066E50B25E0FEE42476
:1002030003FFEE3420FE1208F0EF655A7051E50B40
:1002130025E0FEE42400FFEE3420FE1209587FC0DF
:100223001209307F431209B77FC11209307F4C1284
:1002330009B77FC21209307F451209B77FC312097C
:10024300307F4F1209B77FC41209307F201209B7DC
:100253007FC51209307F4B1209B712092780160593
:100263000BE50B7002050AC39408E50A64809480C9
:1002730050030201BA20B65D7F647E001208D320CA
:10028300B6537F007E201209587F007E2212095840
:100293007F007E241209587F007E261209587F00B2
:1002A3007E281209587F007E2A1209587F007E2C6F
:1002B3001209587F007E2E1209587FC01209307F21
:1002C3004F1209B77FC11209307F4B1209B77F6400
:0502D3007E0012092B62
:0102D8002203
:10045300E4F508F509FB7A0079367F521206E0EFDE
:100463006003020558FB7A007957120665EF6003B3
:100473000205587F801209307F431209B77F81122A
:1004830009307F411209B77F821209307F52120966
:10049300B77F831209307F441209B7E4F508F509E1
:1004A300E50925E0FEE42400FFEE3420FE1208F007
:1004B300EF65576003020542E50925E0FEE42401E8
:1004C300FFEE3420FE1208F0EF65587072E509253F
:1004D300E0FEE42402FFEE3420FE1208F0EF65593B
:1004E300705DE50925E0FEE42403FFEE3420FE12EF
:1004F30008F0EF655A70487F84120930AF5712092C
:10050300B77F85120930AF581209B77F86120930B9
:10051300AF591209B77F87120930AF5A1209B77F53
:10052300C01209307F4F1209B77FC11209307F4BC8
:100533001209B77FF47E011208D37F010209300547
:1005430009E50970020508C39408E50864809480EE
:0505530050030204A3A7
:010558002280
:1008B000758921759840758DE8858D8B758780D2F7
:1008C000AFD2ACD28E1207D21209DC1209947F414A
:0308D000020745D7
:1009A6007580FFC290D291C2A5D2A52087F5C2A5B7
:0109B600221E
:1009B7001209A6C2A58F80D290C291D2A5C2A52244
:090927007FF47E011208D37F0168
:100930001209A6C2A58F80C290C291D2A5C2A522DB
:10096E007F381209307F0C1209307F061209307F52
:04097E000102093039
:0806E0008F0C8B0D8A0E890FAF
:1006E8001209827D077F0D1208107D037F141209FD
:1006F800C7850C12752901752A00752B00752C12F7
:10070800752D00752E00752F107B007A0079127FE9
:100718000C1202D9EF7023E51164104510701BAB61
:100728000DAA0EA90FE512120612AB0DAA0EA90FFB
:0C073800900001E51312062480027FFEF1
:010744002292
:060665008B0C8A0D890ECA
:10066B00E4F510120982E4FD7F0D1208107D807FE6
:10067B000E120986751393751420752902752A00BD
:10068B00752B00752C13752D00752E00752F117B96
:10069B00007A0079137F0C1202D98F0FE50F702BA4
:1006AB00FF74132FF8E6AB0CAA0DA90E8F8275837E
:1006BB000012062474132FF8E662100FBF04E274C5
:1006CB00132FF8E665106003750FFE7D807F0E1209
:0406DB0009C7AF0F8D
:0106DF0022F8
:1007D200D2A000C2A000D2A0007D0F7F011208109B
:1007E200007D3D7F111208107D1E7F2D120810E43E
:1007F200FD7F2C1208107D8D7F2A1208107D3E7F0E
:0E0802002B1208107D407F151208107F002277
:10074500EF6441703F1209827D3D7F111208107DD3
:10075500867F171208107D7F7F261208107D1E7F69
:100765002D120810E4FD7F2C1208107D8D7F2A12B2
:1007750008107D3E7F2B120810E4FFFE12090C12B3
:0A078500099480037FFF227F002209
:06078F00AC07AB05E4FE1F
:10079500E4FEC292C2A4EF25E0547E4480FF7D08AA
:1007A500EF30E703D38001C392A2D292EF25E0FF99
:1007B500C292DDEC7D08D292EE25E0FEA2A1E433E3
:0C07C5004206C292DDF0D2A4D292AF0630
:0107D1002205
:10081000C292C2A4EF25E0547EFF7E08EF30E703CA
:10082000D38001C392A2D292EF25E0FFC292DEEC08
:100830007E08ED30E703D38001C392A2D292ED256A
:0A084000E0FDC292DEECD2A4D292D9
:01084A00228B
:0D09C70012078FAE07AF04EB4EFD020810C3
:040982007D087F0865
:0E09860012078FAE07AF04EBF45EFD020810FF
:0802D9008F258B268A27892856
:1002E1007530FEE4F531F532E52524F4600C24FE89
:1002F100700E753112753210800675317775323096
:10030100E5314480FD7F021208107D807F041209CF
:1003110086E4FD7F011208107D807F0A1209C7E47F
:10032100F534F535C3E5359529E5349400501FAB17
:1003310026AA27A9288535828534831205E5FD7F04
:10034100091208100535E53570DA053480D6AD257A
:100351007F01120810E525B40C077D807F0D12097D
:10036100C77534077535D07F041207958F33E5358E
:10037100153570021534E53545346009E53320E063
:1003810004553260E27D807F0D120986E5354534E2
:1003910070030204427F06120795EF541B600302AB
:1003A100043FF530E533553130E0037530FFE52585
:1003B100640C60030204427F0A1207958F337F0C9D
:1003C100120795EF5407FD6021E53324FFFFE43464
:1003D100FFFEEF7803C333CE33CED8F97C002DFF77
:1003E100EC3EAB2DAA2EA92F800FE53375F008A4A2
:1003F100FFAB2DAA2EA92FE5F08FF0120646E533AB
:100401007003753301E533D394124003753312E45D
:10041100F534F535C3E5359533E534940050227F45
:1004210009120795AB2AAA2BA92C8535828534831D
:10043100EF1206240535E53570DA053480D67530BE
:10044100FE7D807F0C1209C7E4FD7F01120810AF09
:01045100307A
:010452002287
:100994007F14120795EF540370077D037F14120927
:0109A400C78B
:0109A500222F
:0709DC007D037F1402098670
:10090C00E4F5CAF5CCD2CAEF1FAC0670011E4C60E0
:0B091C000730CFFDC2CF80EFC2CA221F
:1009580075E78175E5038FE48EE3C2AF75E64675EA
:06096800E6B9000209D40B
:1009400075E78175E5028FE48EE38DE2C2AF75E64F
:080950004675E6B9000209D466
:1008F00075E78175E5018FE48EE3C2AF75E6467555
:0B090000E6B90085E20C1209D4AF0C30
:01090B0022C9
:0809D400E4F5E7F5E5F5E62284
:1005650002084BE493A3F8E493A34003F68001F259
:1005750008DFF48029E493A3F85407240CC8C33397
:10058500C4540F4420C8834004F456800146F6DF66
:10059500E4800B0102040810204080900881E47E6D
:1005A500019360BCA3FF543F30E509541FFEE4935B
:1005B500A360010ECF54C025E060A840B8E493A322
:1005C500FAE493A3F8E493A3C8C582C8CAC583CA4D
:1005D500F0A3C8C582C8CAC583CADFE9DEE780BE05
:0108AF000048
:1005E500BB010CE58229F582E5833AF583E02250CB
:1005F50006E92582F8E622BBFE06E92582F8E22215
:0D060500E58229F582E5833AF583E493222E
:10061200BB010689828A83F0225002F722BBFE01C7
:02062200F322C1
:10062400F8BB010DE58229F582E5833AF583E8F00C
:10063400225006E92582C8F622BBFE05E92582C8B8
:02064400F222A0
:10064600BB010A89828A83F0E5F0A3F0225006F7FF
:0F06560009A7F01922BBFE06F3E5F009F31922FC
:00000001FF
